:020000040800F2
:1000000000500020554700088108000889080008B2
:100010008B0800088D0800088F0800080000000009
:10002000000000000000000000000000910800082F
:1000300093080008000000009508000897080008D1
:100040009D4700089D4700089D4700089D47000800
:100050009D4700089D4700089D4700089D470008F0
:100060009D4700089D4700089D4700089D470008E0
:100070009D4700089D4700089D4700089D470008D0
:100080009D4700089D4700089D4700089D470008C0
:10009000990800089D4700089D4700089D470008F3
:1000A0009D4700089D4700089D4700089D470008A0
:1000B0009D4700089D470008A90800089D470008C3
:1000C0009D4700089D4700089D4700089D47000880
:1000D0009D4700089D4700089D4700089D47000870
:1000E0009D4700089D4700089D470008000000004C
:1000F0000000000000000000000000000000000000
:0C01000000000000000000005FF808F1A3
:10010C00034613F8012B002AFBD1181A013870474B
:10011C0010B5054C237833B9044B13B10448AFF335
:10012C0000800123237010BD10020020000000008D
:10013C00BC50000808B5034B1BB103490348AFF38F
:10014C00008008BD0000000014020020BC50000814
:10015C0038B50446836801210068984763680A2112
:10016C0020689847A36800212068984763684FF47B
:10017C00F07120689847A36801212068984763684C
:10018C00462120689847E3682068984705466368CD
:10019C004FF4CD7120689847B5FA85F0400938BD09
:1001AC0038B50446836800210068984763680621C7
:1001BC0020689847A3680121206898476368092143
:1001CC0020689847E368206898470546636837219C
:1001DC0020689847284638BD70B504460E46002561
:1001EC0012E0A36800212068984763683C212068CE
:1001FC009847A36801212068984763680A21206802
:10020C00984776080135EDB2072D13D816F0010F7B
:10021C00E7D0A3680021206898476368062120680E
:10022C009847A3680121206898476368402120689B
:10023C009847E6E7002070BDF8B5044600252F4628
:10024C0001E00135EDB2072D1ED87F08A36800210F
:10025C00206898476368062120689847A3680121A5
:10026C00206898476368092120689847E3682068EC
:10027C00984706466368372120689847002EE0D0DF
:10028C0067F07F07FFB2DCE73846F8BD034602781B
:10029C004A400249885C1870704700BFD45000086F
:1002AC002DE9F04F83B00446019100230377D0F879
:1002BC0018B0BBF1000F07D000232361A361636169
:1002CC00012003B0BDE8F08FFFF742FF28B90023EF
:1002DC002361A36163610120F3E7F0212046FFF75E
:1002EC007BFFD8460126B14653E0012F40F08580B4
:1002FC00B9F1400FE0DD207F0028DDD1C4F810B04B
:10030C00BBF1000F01D10123A361637F002BD3D07C
:10031C00D4F81D20D4F8213001990A604B60D0E745
:10032C0025694D450FDD04EB08035B7F334214BF99
:10033C0001250025002D62D1B9F1080F08DCC4F8A5
:10034C001490CB465BE04D4514BF00250125F1E729
:10035C00CB4654E004EB0802537F3343537757E00A
:10036C00A36800212068984763683C21206898475F
:10037C00A36801212068984763680A212068984780
:10038C0009F10109760016F0FF0654D0B8F1070FF9
:10039C00AEDCA368002120689847636806212068BA
:1003AC009847A36801212068984763680921206851
:1003BC009847E368206898470546636837212068AA
:1003CC009847AA46A36800212068984763680621CD
:1003DC0020689847A3680121206898476368092121
:1003EC0020689847E3682068984707466368372178
:1003FC0020689847012D3FF478AFBA4590D0012D75
:10040C00A8D0F24352B204EB08014B7F13404B7758
:10041C00002DA5D0A36800212068984763680621A9
:10042C0020689847A3680121206898476368402199
:10043C0020689847A4E704EB0803597F04F11C00DB
:10044C00FFF724FF08F1010801269FE7034600206F
:10045C00186198615861704708B5FFF721FF08BD16
:10046C00052901D80020704710B584B00C466846A9
:10047C0003F0C6FA053C019B0E4AA2FB03239B0C1E
:10048C0003FB04F44FF0E02304221A615C610022A8
:10049C009A611A6942F001021A614FF0E0231B695C
:1004AC0013F4803FF9D04FF0E02304221A610020AE
:1004BC0004B010BD83DE1B4331B102684368C3F343
:1004CC000F2313610020704702684368C3F30F23A6
:1004DC005361F7E7026843689068C04300EA132051
:1004EC0080B2B0FA80F04009704738B50546552106
:1004FC000068FFF771FE002406E02B1919792868B3
:10050C00FFF76AFE0134E4B2072CF6D9002038BD9F
:10051C0010B504460068FFF71BFE2046FFF7E5FF09
:10052C0044212068FFF758FE002010BD08B5006874
:10053C00FFF736FE08B9012008BD0020FCE70000DB
:10054C0038B505460C460068FFF702FE2846FFF753
:10055C00CCFFBE212868FFF73FFE2868FFF76CFE32
:10056C0060702868FFF768FE20702868FFF7F0FDC0
:10057C00237813F0F80F16D00C4A62801B0203F498
:10058C00E0631343638062781343638040F271220B
:10059C0002FB03F3064A82FB0312DB17C3EBA21325
:1005AC006380002038BD0022E7E700BF0080FFFF1A
:1005BC00D34D6210F0B589B00024049405940694D0
:1005CC000794214B9A6942F020029A619A6902F0D1
:1005DC0020020192019A9A6942F004029A619A6986
:1005EC0002F004020292029A9A6942F008029A619D
:1005FC009B6903F008030393039B144F22464FF4AB
:10060C000071384602F0E2FF114D01224FF4807167
:10061C00284602F0DBFF4FF4007304930126059685
:10062C0006940224079404A9384602F03BFE4FF4CA
:10063C0080730493112305930696079404A9284606
:10064C0002F030FE09B0F0BD00100240000801407D
:10065C00000C0140F0B587B000240294039404947C
:10066C000594154DAB6943F00403AB61AB6903F022
:10067C0004030193019B114E22464FF480513046E6
:10068C0002F0A4FF4FF480570297012303930494C4
:10069C000223059302A9304602F004FE642002F006
:1006AC0009FA3946304602F00FFFAB6923F0040318
:1006BC00AB6107B0F0BD00BF001002400008014064
:1006CC0008B50268034B9A4200D008BD02F0E0F96D
:1006DC00FBE700BF0008004072B6FEE708B507480C
:1006EC00074B03600523436040F6FF73836003F000
:1006FC00FFFF00B908BDFFF7EFFF00BF2C02002081
:10070C000030004000B595B0282200210DEB02000E
:10071C0004F064F800230593069307930893099358
:10072C00019302930393049309230A934FF48033A8
:10073C000B9301220E9210920222119212934FF4FB
:10074C00E01313930AA802F0DFF9D0B90F23059335
:10075C0002210691002307934FF4806208920993BB
:10076C0005A802F017FC70B9102301930023049321
:10077C0001A802F00BFD40B902F0CEFB15B05DF8FC
:10078C0004FBFFF7A9FFFFF7A7FFFFF7A5FF00008A
:10079C0080B5CEB002F06AF9FFF7B4FFFFF75AFF4D
:1007AC00FFF708FF00F0E2F8FFF798FF2D4C20460A
:1007BC00FFF7CEFC002349934A934B9349944CE0AA
:1007CC000A2002F077F949A8FFF7B0FE0028F7D10C
:1007DC0048A949A8FFF7B4FE9DF831319DF83221A4
:1007EC009DF833119DF834019DF835419DF8365133
:1007FC009DF83761BDF9227107970696059504940B
:10080C0003900291019200939DF83031164AFF211A
:10081C0008A803F0EBFF08A8FFF772FC81B208A848
:10082C0000F08EF9114803F088FF4CA90D48FFF732
:10083C0013FE012809D04AAB4EAA12E9030083E843
:10084C00030049A8FFF764FEBDE74FF400710848A8
:10085C0002F0C2FE642002F02DF90248FFF7F6FD0B
:10086C00E3E700BF00000020D45100082C02002058
:10087C000008014008B502F079FCFEE7FEE7FEE750
:10088C00FEE7FEE7704770477047704708B50248AF
:10089C0000F053FF08BD00BF140F002008B502483C
:1008AC0002F036FF08BD00BF3802002082B00E4BAC
:1008BC009A6942F001029A619A6902F0010200926F
:1008CC00009ADA6942F08052DA61DB6903F08053F6
:1008DC000193019B054A536823F0E06343F00073D6
:1008EC00536002B0704700BF00100240000001408E
:1008FC0000B589B0014600221E2002F089FE1E20A0
:10090C0002F0BEFE154BDA6942F00402DA61DB69D3
:10091C0003F004030193019B02A903A802F006FC57
:10092C0002F0F4FB43000E4AA2FB03239B0C013B99
:10093C000C480D4A026040F2E732C260436000236B
:10094C000361836002F0DCFF18B1012009B05DF88F
:10095C0004FB044802F0A4FEF8E700BF00100240BC
:10096C0083DE1B43380200200008004008B500223B
:10097C000F49104803F055F870B90F490D4803F0B2
:10098C0067F860B90D490B4803F06BFE50B9094884
:10099C0003F065F848B908BDFFF79EFEEDE7FFF7D9
:1009AC009BFEEFE7FFF798FEF1E7FFF795FEF2E706
:1009BC0030000020800200209C00002080000020DD
:1009CC0012230B80004870474C00002004230B803E
:1009DC000048704760000020002393421ED200B5EF
:1009EC0010E00CF1370C01F813C000014FEA430C76
:1009FC000CF1010C4FF0000E01F80CE00133DBB2EE
:100A0C00934209D24FEA107CB0F1204FE9D20CF19D
:100A1C00300C01F813C0E8E75DF804FB70470000E8
:100A2C0038B50B4BD3F8E807D3F8EC47D3F8F037CD
:100A3C00C01800D138BD074D0822A91CFFF7CCFF08
:100A4C00042205F112012046FFF7C6FFF2E700BFB2
:100A5C0000F0FF1F6400002008B51A230B80FFF77D
:100A6C00DFFF014808BD00BF6400002008B50A463E
:100A7C0028B90549054803F04AFC034808BD02495A
:100A8C00024803F044FCF8E744050020FC51000840
:100A9C0010B50A46034C2146034803F038FC2046A7
:100AAC0010BD00BF440500201452000808B50A46CA
:100ABC0028B90549054803F02AFC034808BD02493A
:100ACC00024803F024FCF8E74405002028520008F3
:100ADC0008B50A4628B90549054803F018FC03482F
:100AEC0008BD0249024803F012FCF8E74405002057
:100AFC0034520008002070470020704710B50146A2
:100B0C00044C204603F0BCFD204603F0D9FD002028
:100B1C0010BD00BF8002002010B5064C0022064913
:100B2C00204603F0A5FD0549204603F0A9FD002051
:100B3C0010BD00BF800200202C0B002044070020B9
:100B4C00094BD3F8B832D3F814320BB101207047EB
:100B5C0010B5054C0A460146204603F089FD204697
:100B6C0003F094FD10BD00BF80020020022805D8C0
:100B7C00DFE800F0050402000120704702207047F6
:100B8C0002680E4B9A4200D0704700B583B003F553
:100B9C00DA33DA6942F40002DA61DB6903F4000348
:100BAC000193019B00221146142002F031FD142008
:100BBC0002F066FD03B05DF804FB00BF005C004072
:100BCC0008B500F52C71D0F8E80202F060FF08BD02
:100BDC0008B501EB810300EBC303D3F87C21D0F8FB
:100BEC00E80202F081FF08BD08B501EB810300EBC0
:100BFC00C303DA6BD0F8E80202F0BCFF08BD08B5FD
:100C0C00D0F8E80203F05DF808BD10B5044683681F
:100C1C00022B09D10121D4F8E80203F03BF8D4F8F7
:100C2C00E80203F00FF810BDFFF756FDF2E70000E5
:100C3C0010B50446D0F8E80203F02FF8A36923B1ED
:100C4C00024A136943F00603136110BD00ED00E086
:100C5C0008B5D0F8E80203F029F808BD10B5044631
:100C6C001D48C0F8E842C4F8C0021C4B03600823BE
:100C7C0043600223836000238361C361036200F03D
:100C8C0023F930BB182300221146D4F8C00200F01F
:100C9C007CFF582300228021D4F8C00200F075FF9D
:100CAC00C02300228121D4F8C00200F06EFF4FF463
:100CBC00887300220121D4F8C00200F066FF4FF4C3
:100CCC00807300228221D4F8C00200F05EFF002065
:100CDC0010BDFFF701FDD5E7140F0020005C0040AC
:100CEC0008B5D0F8C00200F07BF9FFF73FFF08BD54
:100CFC0008B594461A466346D0F8C00200F007FEC9
:100D0C00FFF734FF08BD08B5D0F8C00200F041FE73
:100D1C00FFF72CFF08BD08B5D0F8C00200F0BEFEEE
:100D2C00FFF724FF08BD08B5D0F8C00200F0F2FEB2
:100D3C00FFF71CFF08BDD0F8C03211F0800F08D1AE
:100D4C0001F07F0101EB810103EBC10393F86A0110
:100D5C00704701F07F01013101EB810103EBC1030D
:100D6C009878704708B5D0F8C00200F0D2FCFFF7B5
:100D7C00FDFE08BD08B5D0F8C00200F067FEFFF715
:100D8C00F5FE08BD08B5D0F8C00200F034FEFFF740
:100D9C00EDFE08BD08B5D0F8C00200F04EFE08BD4F
:100DAC0000487047001200207047704738B512F4A5
:100DBC00804F44D00468B4F850309BB291F800C016
:100DCC0003EBCC03023304EB4304B4F80044C4F348
:100DDC0009048B69A34228D31B1B8B618B697BB9DC
:100DEC00056835F82C309BB223F4804323F0700354
:100DFC0083F4005343F4004343F0800325F82C3074
:100E0C0012F0400F0ED002680D7832F825309BB2EC
:100E1C0023F4E04323F0700343F4004343F0C00396
:100E2C0022F8253024B9204638BD00238B61D5E744
:100E3C0023460A894969006801F0FFFDF3E704685D
:100E4C00B4F850309BB291F800C003EBCC030633DE
:100E5C0004EB4304B4F80044C4F309048B69A342C3
:100E6C002FD31B1B8B618B697BB9056835F82C3034
:100E7C009BB223F4804323F0700383F4005343F4B8
:100E8C00004343F0800325F82C3012F0400F0FD1B3
:100E9C00026891F800C032F82C309BB223F4E04386
:100EAC0023F0700343F4004343F0C00322F82C30CA
:100EBC00002CB8D023464A894969006801F0BDFD71
:100ECC00B1E700238B61CEE770B586B0002800F047
:100EDC008580044690F8A932EBB1032384F8A9323B
:100EEC00206800F07EFE254655F8106BEC460FCDC1
:100EFC00ACE80F002B68CCF80030231D0ECB30462D
:100F0C0000F05FFE054658B1022384F8A932012592
:100F1C00284606B070BD80F8A832FFF731FEDCE73A
:100F2C000021206800F067FE2B461AE05A1C02EBE9
:100F3C00820104EBC1010120487002EB820104F82C
:100F4C00313003EB830104EBC101CB8602EB820C45
:100F5C0004EBCC0C00208CF803008863C863086495
:100F6C00D3B261688B42E1D316E005EB850304EB49
:100F7C00C303002283F8692183F8685183F86B213D
:100F8C00C3F87821C3F87C2105EB850304EBC3037C
:100F9C00C3F880210135EDB2A942E6D8254655F8B3
:100FAC00106BEC460FCDACE80F002B68CCF8003082
:100FBC00231D0ECB304600F020FE054620B1022347
:100FCC0084F8A9320125A3E7002384F824300123F7
:100FDC0084F8A932206801F046F999E7012597E7D2
:100FEC0038B590F8A832012B11D00446012580F8B1
:100FFC00A852006800F0ECFD29462046FFF7D5FE0C
:10100C00206801F02EF9002084F8A80238BD0220D7
:10101C00FCE770B505460C46164612F0400F00F082
:10102C00BA800268B2F850309BB2097803EBC10366
:10103C00023302EB4302B2F80024C2F30902A369A3
:10104C0093422BD99B1AA361A36953B316F4804F17
:10105C000DD0286830F821309BB223F4E04323F004
:10106C00700343F4404343F0800320F8213094F89C
:10107C002430012B2BD02A68217832F821309BB2F6
:10108C0023F4E04323F0400383F0300343F40043A4
:10109C0043F0800322F82130002070BD0023A361AF
:1010AC00D2E72846FFF7A0FD16F4804FE3D02A685C
:1010BC00217832F821309BB223F4E04323F0700303
:1010CC0043F4404343F0800322F82130D3E76369B3
:1010DC0013446361E3691344E361216A2369994210
:1010EC001FD3C91A21626278002A3FD12A68B2F84C
:1010FC00501089B20A44217802EB0112EBB9B2F814
:10110C00041489B221F4F84189B2A2F80414B2F89B
:10111C0004146FEA41416FEA514189B2A2F80414F8
:10112C0026E021B9002384F824301346DBE70023A2
:10113C0084F8243023620B46D5E73E2B09D8590896
:10114C0013F0010F00D00131890289B2A2F8041406
:10115C000EE0590913F01F0F00D101396FEAC1617C
:10116C006FEA514189B2A2F8041401E0012A06D0B9
:10117C009BB222896169286801F07DF87BE72A68B7
:10118C00B2F8501089B20A44217802EB011299B2DC
:10119C00A2F80414ECE70268B2F850309BB209785C
:1011AC0003EBC103063302EB4302B2F80024C2F393
:1011BC000902A369934244D39B1AA361A369002B30
:1011CC0042D016F4804F0DD1286830F821309BB2F4
:1011DC0023F4E04323F0700343F4404343F08003D3
:1011EC0020F8213094F82430012B7FF444AF63694C
:1011FC0013446361E3691344E361216A23699942EF
:10120C0039D3C91A21622A686178002958D1B2F8F9
:10121C00501089B20A44217802EB0112BBBBB2F820
:10122C000C1489B221F4F84189B2A2F80C14B2F86A
:10123C000C146FEA41416FEA514189B2A2F80C14C7
:10124C0040E00023A361B9E72846FFF7CDFC16F474
:10125C00804F7FF410AF2A68217832F821309BB28E
:10126C0023F4E04323F0700343F4404343F0800342
:10127C0022F82130FFE621B9002384F824301346EC
:10128C00C1E70023236284F824300B46BBE73E2BD6
:10129C0009D8590813F0010F00D00131890289B225
:1012AC00A2F80C140EE0590913F01F0F00D10139EC
:1012BC006FEAC1616FEA514189B2A2F80C1401E0E6
:1012CC00012906D09BB262896169286800F0D3FFBE
:1012DC00D1E6B2F8501089B20A44217802EB01121F
:1012EC0099B2A2F80C14EDE72DE9F04105462868F7
:1012FC00B0F8443013F4004F00F00882B0F84440CA
:10130C00A3B214F00F0440F0D48013F0100F5DD092
:10131C0003889AB213F4006F40F08F8012F4004FE0
:10132C00E5D0038823F070031B051B0D43F08003ED
:10133C0003802868B0F850309BB295F8682103EB15
:10134C00C203063300EB4303B3F80034C3F30903C1
:10135C00C5F884318BB1D5F87C1171B1B5F86E211B
:10136C0001F06BFBD5F88421D5F87C311344C5F81A
:10137C007C3100212846FFF72BFC2B68B3F850205A
:10138C0092B21344D5F87821002A79D1B3F80C2401
:10139C0092B222F4F84292B2A3F80C24B3F80C24C3
:1013AC006FEA42426FEA524292B2A3F80C242A68C6
:1013BC0013889BB223F4804323F0700383F44053CF
:1013CC0043F4004343F08003138090E703889BB2FF
:1013DC0023F4E14323F070036FEA43436FEA534372
:1013EC009BB203802A68B2F850309BB295F8281053
:1013FC0003EBC103023302EB4302B2F80034C3F334
:10140C0009036B64EA6B1A44EA6300212846FFF770
:10141C00EBFB95F82430002B3FF469AF2B6C002BC1
:10142C007FF465AF95F824302A6843F08003A2F866
:10143C004C30002385F8243059E7B0F850309BB27B
:10144C0095F8682103EBC203063300EB4303B3F8B2
:10145C000034C3F30903C5F88431B5F86E2105F5E2
:10146C002C7101F0EAFA2A68138823F070031B052B
:10147C001B0D43F0800313802846FFF7A1FB36E7D2
:10148C003E2A09D8510812F0010F00D0013189020F
:10149C0089B2A3F80C148AE7510912F01F0F00D17E
:1014AC0001396FEAC1626FEA524292B2A3F80C247E
:1014BC007DE730F824309EB213F4004F48D116F07B
:1014CC00800F3FF414AF621C02EB820105EBC101EB
:1014DC00286830F824309BB223F4E14323F07003E6
:1014EC006FEA43436FEA53439BB220F82430CB7826
:1014FC00022B00F0EE802868B0F850309BB2621CD2
:10150C0002EB820215F8326003EBC603023300EBE8
:10151C004303B3F80034C3F3090304EB840205EB73
:10152C00C202126C9A4240F2DD8004EB840705EB98
:10153C00C707D21A3A6404EB840205EBC202126CA0
:10154C00002A40F0D68031462846FFF74DFBCEE608
:10155C0030F8243023F070031B051B0D43F080037F
:10156C0020F8243004EB8401C90001F5B47105EBBB
:10157C00010804EB840305EBC30393F87431002BCF
:10158C0042D12868B0F850309BB204EB840205EBD2
:10159C00C20292F8682103EBC203063300EB43034B
:1015AC00B3F80074C7F3090717BB04EB840305EB0E
:1015BC00C303D3F884213A44C3F88421D3F87C21A3
:1015CC003A44C3F87C21D3F880313BB104EB84035B
:1015DC0005EBC303D3F878319F4275D204EB840337
:1015EC0005EBC30393F868112846FFF7F1FA66E799
:1015FC0004EB840105EBC1013B46B1F86E21D1F837
:10160C007C1101F01AFAD0E704EB840305EBC30359
:10161C0093F86B31022B35D0296804EB840205EB6F
:10162C00C20292F8680131F820309BB223F4E043F7
:10163C0023F0700343F4004343F0C00321F820303F
:10164C00286892F8682130F8223013F4804F20D0AB
:10165C00B0F850309BB203EBC203023300EB4303F0
:10166C00B3F80074C7F30907002F9ED004EB840174
:10167C0005EBC1013B46B1F87021D1F87C1101F0AA
:10168C00DCF992E7324641462846FFF78FFB0746C6
:10169C008BE7B0F850309BB203EBC203063300EB80
:1016AC004303B3F80074C7F30907002F3FF47DAF71
:1016BC0004EB840105EBC1013B46B1F87221D1F872
:1016CC007C1101F0BAF970E74146286800F0E6FD9C
:1016DC00F5E616F4807F3FF40EAF32462846FFF74E
:1016EC0098FC04E604EB840205EBC20200271764A5
:1016FC0021E704EB840205EBC202D66B1E44D663D1
:10170C00546C2344536400F0C9FDF0E50020BDE89F
:10171C00F08190F8A832012B0DD010B504460123AE
:10172C0080F8A83280F82410006800F094FD0020A6
:10173C0084F8A80210BD0220704710B584B004468E
:10174C00006800F092FD10F4004F47D1206800F0C3
:10175C008CFD10F4806F45D1206800F086FD10F4EC
:10176C00804F08D02268B2F844309BB223F48043F7
:10177C009BB2A2F84430206800F077FD10F4005FB3
:10178C0008D02268B2F844309BB223F400539BB2C9
:10179C00A2F84430206800F068FD10F4805F32D16C
:1017AC00206800F062FD10F4006F78D1206800F022
:1017BC005CFD10F4007F40F09D80206800F055FD2A
:1017CC0010F4807F08D02268B2F844309BB223F426
:1017DC0080739BB2A2F8443004B010BD2046FFF7D2
:1017EC0083FDB3E72268B2F844309BB223F48063E4
:1017FC009BB2A2F844302046FFF707FA002120469E
:10180C00FFF787FFA8E72268B2F840309BB223F0BD
:10181C0004039BB2A2F840302268B2F840309BB26D
:10182C0023F008039BB2A2F840302046FFF710FAD1
:10183C002268B2F844309BB223F480539BB2A2F8D6
:10184C004430ADE7226832F8231004AA02EB4302BD
:10185C0022F8101C0133DBB2072BF3D92268B2F843
:10186C0040309BB243F00103A2F840302268B2F83A
:10187C0040309BB223F001039BB2A2F840302368A6
:10188C00B3F8442012F4806FF9D0B3F8442092B22C
:10189C0022F4806292B2A3F8442000230BE00023D0
:1018AC00DAE7226804A901EB430131F8101C22F895
:1018BC0023100133DBB2072BF3D92268B2F8403086
:1018CC009BB243F00803A2F840302268B2F84430CF
:1018DC009BB223F400639BB2A2F844302268B2F8A6
:1018EC0040309BB243F00403A2F840302046FFF78F
:1018FC009FF95BE72268B2F844309BB223F4007383
:10190C009BB2A2F844302046FFF779F955E710B5A1
:10191C0004468C4611F0800F2AD101F0070000EB31
:10192C008001C90001F5B47E04EB0E0100EB8000D0
:10193C0004EBC0004FF0000E80F869E10CF0070CCE
:10194C0081F800C00A61CB704A780AB1A1F80EC0C8
:10195C00022B19D094F8A832012B18D0012384F84B
:10196C00A832206800F05AF9002084F8A80210BDB3
:10197C0001F00700013000EB800104EBC1014FF0D6
:10198C00010E81F801E0D9E700230B71E2E7022098
:10199C00EDE710B504460B4611F0800F1FD101F096
:1019AC00070202EB8201C90001F5B471014402EB9C
:1019BC00820200EBC202002082F8690103F00703E7
:1019CC000B7094F8A832012B13D0012384F8A832A1
:1019DC00206800F0DFFA002084F8A80210BD01F0A6
:1019EC000702013202EB820100EBC10101204870B9
:1019FC00E4E70220F2E710B501F0070404EB8401E0
:101A0C00C90001F5B471014404EB840C00EBCC0C5F
:101A1C00CCF87C21CCF880310023CCF884318CF8C4
:101A2C0069318CF8684124B9006800F037FC00205B
:101A3C0010BD006800F032FCF9E701F0070101EB82
:101A4C00810100EBC100D0F88401704710B501F0A2
:101A5C00070404F1010C0CEB8C0100EBC10104EB4D
:101A6C00840E00EBCE0ECEF83C20CEF84030012296
:101A7C008EF84C20CEF848300023CEF844304A7013
:101A8C000CEB8C0C00F83C4024B9006800F006FC10
:101A9C00002010BD006800F001FCF9E738B501F03A
:101AAC0007054268954231D804460B4611F0800F69
:101ABC001ED101EB8101C90001F5B471014403EBA6
:101ACC00830300EBC303002283F8692101238B708D
:101ADC000D7094F8A832012B1AD0012384F8A83287
:101AEC00206800F042FB5DB1002084F8A80238BDEC
:101AFC006B1C03EB830100EBC10101224A70E5E78B
:101B0C0004F52C71206800F0B4FBEDE70120EEE742
:101B1C000220ECE70B4601F00F014268914230D8ED
:101B2C0010B5044613F0800F21D103F0070202EB2D
:101B3C008201C90001F5B471014402EB820200EB91
:101B4C00C202002082F8690100228A7003F00703A8
:101B5C000B7094F8A832012B15D0012384F8A8320D
:101B6C00206800F027FB002084F8A80210BD03F0C9
:101B7C000702013202EB820100EBC1010120487027
:101B8C00E2E7012070470220F0E711F0800F0BD044
:101B9C0001F00701013101EB810100EBC10052B9E9
:101BAC000273C3800020704701EB8101C90001F56D
:101BBC00B4710844F3E70122027303811B0C4381C7
:101BCC00F0E784B001A880E80E00002004B0704754
:101BDC0003460020A3F844004FF43F42A3F84020F2
:101BEC007047B0F8403023F47C535B045B0CA0F8D6
:101BFC004030002070470020704784B0844601A814
:101C0C0080E80E000123ACF840300020ACF8400016
:101C1C00ACF84400ACF8500004B0704710B5034663
:101C2C0091F800C030F82C2092B222F4EC4222F051
:101C3C00700292B2C878032861D8DFE800F0555CD6
:101C4C000258002048F2800E42EA0E0223F82C20A3
:101C5C0091F800C033F82C2092B222F4E04222F02A
:101C6C0070024CEA020242EA0E0223F82C200A7B94
:101C7C00002A40F0C4804A78002A51D0B3F8502092
:101C8C0092B21A440C7802EB0412B1F806C04FEA77
:101C9C005C0C4FEA4C0CA2F800C40C7833F82420EE
:101CAC0012F0400F0CD033F8242092B222F4E04210
:101CBC0022F0700242F4004242F0C00223F82420C9
:101CCC00CA78012A1DD0097833F8212092B222F467
:101CDC00E04222F0400282F0200242F4004242F044
:101CEC00800223F821206AE042F40072AAE742F451
:101CFC00C0620020A6E742F480620020A2E7012027
:101D0C00A0E7097833F8212092B222F4E04222F0C5
:101D1C00400242F4004242F0800223F821204EE0BF
:101D2C00B3F8502092B21A440C7802EB0412B1F8BA
:101D3C0006C04FEA5C0C4FEA4C0CA2F808C4B3F88E
:101D4C00502092B21A440C7802EB04120C69BCBB02
:101D5C00B2F80CC41FFA8CFC2CF4F84C1FFA8CFC57
:101D6C00A2F80CC4B2F80CC46FEA4C4C6FEA5C4C91
:101D7C001FFA8CFCA2F80CC40C7833F8242012F453
:101D8C00804F0CD033F8242092B222F4E04222F09F
:101D9C00700242F4404242F0800223F82420097879
:101DAC0033F8212092B222F4804222F0700282F4A5
:101DBC00405242F4004242F0800223F8212010BD30
:101DCC003E2C0DD84FEA540C14F0010F01D00CF13D
:101DDC00010C4FEA8C2C1FFA8CFCA2F80CC4CBE73C
:101DEC004FEA541C14F01F0F01D10CF1FF3C6FEAA9
:101DFC00CC646FEA5444A4B2A2F80C44BCE791F84A
:101E0C0000C033F82C2092B222F4E04222F070028F
:101E1C0042F4014242F0800223F82C20B3F8502007
:101E2C0092B21A4491F800C002EB0C12B1F808C03F
:101E3C004FEA5C0C4FEA4C0CA2F800C4B3F85020EB
:101E4C0092B21A4491F800C002EB0C12B1F80AC01D
:101E5C004FEA5C0C4FEA4C0CA2F808C44A78002AF2
:101E6C0041D10C7833F8242012F4804F0CD033F885
:101E7C00242092B222F4E04222F0700242F440425A
:101E8C0042F0800223F824200C7833F8242012F03E
:101E9C00400F0CD033F8242092B222F4E04222F00E
:101EAC00700242F4004242F0C00223F8242091F860
:101EBC0000C033F82C2092B222F4804222F070023F
:101ECC0082F4405248F28004224323F82C200978F3
:101EDC0033F8212092B222F4E04222F04002224355
:101EEC0023F821206BE70C7833F8242012F4804F70
:101EFC000CD033F8242092B222F4E04222F070028B
:101F0C0042F4404242F0800223F824200C7833F84B
:101F1C00242012F0400F0CD033F8242092B222F47B
:101F2C00E04222F0700242F4004242F0C00223F878
:101F3C002420CA78012A1ED00C7833F8242092B2BF
:101F4C0022F4E04222F0400282F0200242F40042ED
:101F5C0042F0800223F82420097833F8212092B231
:101F6C0022F4804222F0700242F4004242F08002DD
:101F7C0023F8212023E70C7833F8242092B222F4A2
:101F8C00E04222F0400242F4004242F0800223F888
:101F9C002420E1E70B7B002B46D14B7813B30A7856
:101FAC0030F8223013F0400F0CD030F822309BB2B6
:101FBC0023F4E04323F0700343F4004343F0C003E5
:101FCC0020F822300A7830F822309BB223F4E04318
:101FDC0023F0400343F4004343F0800320F8223005
:101FEC00002070470A7830F8223013F4804F0CD060
:101FFC0030F822309BB223F4E04323F0700343F417
:10200C00404343F0800320F822300A7830F8223025
:10201C009BB223F4804323F0700343F4004343F05A
:10202C00800320F82230DBE74B78002B4ED10A7866
:10203C0030F8223013F4804F0CD030F822309BB2A1
:10204C0023F4E04323F0700343F4404343F0800354
:10205C0020F822300A7830F8223013F0400F0CD0E0
:10206C0030F822309BB223F4E04323F0700343F4A6
:10207C00004343F0C00320F822300A7830F82230B5
:10208C009BB223F4E04323F0700343F4004343F08A
:10209C00C00320F822300A7830F822309BB223F4A7
:1020AC00804323F0700348F2800C43EA0C0320F8C1
:1020BC0022300A7830F822309BB223F4E04323F02C
:1020CC00400343EA0C0320F8223089E70A7830F801
:1020DC00223013F4804F0CD030F822309BB223F412
:1020EC00E04323F0700343F4404343F0800320F8B3
:1020FC0022300A7830F8223013F0400F0CD030F830
:10210C0022309BB223F4E04323F0700343F40043EA
:10211C0043F0C00320F822300A7830F822309BB20A
:10212C0023F4E04323F0700343F4404343F0800373
:10213C0020F822300A7830F822309BB223F4E043A6
:10214C0023F0400348F2800C43EA0C0320F82230C1
:10215C000A7830F822309BB223F4804323F07003CA
:10216C0043EA0C0320F822303AE74B788BB10A781B
:10217C0030F822309BB223F4E04323F0400383F089
:10218C00100343F4004343F0800320F82230002076
:10219C0070470A7830F822309BB223F4804323F046
:1021AC00700383F4805343F4004343F0800320F81E
:1021BC002230ECE70B7B002B4BD14B7833B30A78F6
:1021CC0030F8223013F0400F0CD030F822309BB294
:1021DC0023F4E04323F0700343F4004343F0C003C3
:1021EC0020F82230CB78012B33D00A7830F822300B
:1021FC009BB223F4E04323F0400383F0200343F429
:10220C00004343F0800320F8223022E00A7830F8B3
:10221C00223013F4804F0CD030F822309BB223F4D0
:10222C00E04323F0700343F4404343F0800320F871
:10223C0022300A7830F822309BB223F4804323F00A
:10224C00700383F4405343F4004343F0800320F8BD
:10225C0022300020704711B98023A0F84C300020A8
:10226C0070470020704700207047B0F8440080B2DF
:10227C0070470020704701335B0800EB420000F50B
:10228C00806008E00A7891F801C042EA0C2220F83C
:10229C00042B0231013B002BF4D1704770B505467D
:1022AC000C464A78012A37D00B7B002B40F0A082D9
:1022BC008B690A69934240F27E829B1A8B61B5F856
:1022CC0050309BB22B44217803EB0113002A40F0D1
:1022DC007682B3F80C2492B222F4F84292B2A3F8AC
:1022EC000C24B3F80C246FEA42426FEA524292B2C9
:1022FC00A3F80C24227835F822309BB223F48043C7
:10230C0023F0700383F4405343F4004343F0800301
:10231C0025F82230002070BD8E6909698E4200D9E3
:10232C000E46237B3BB3E378022B46D0217835F85D
:10233C00213013F0400F00F0EE81002A40F0CA81EA
:10234C00B5F850309BB22B4403EB0113002E40F038
:10235C00A881B3F80C2492B222F4F84292B2A3F8FA
:10236C000C24B3F80C246FEA42426FEA524292B248
:10237C00A3F80C24B7E1B6B23346E288616928466B
:10238C00FFF779FFB5F850309BB22B44227803EB62
:10239C000213A3F80464227835F822309BB223F49C
:1023AC00E04323F0400383F0300343F4004343F055
:1023BC00800325F822300020ADE7236A994280F093
:1023CC005281227835F822309BB223F4E04323F07B
:1023DC00700343F4014343F0800325F82230236A51
:1023EC009B1B2362237835F8232012F0400F00F05A
:1023FC009D8062788ABBB5F8502092B22A4402EBD9
:10240C0003138EB9B3F80C2492B222F4F84292B2B0
:10241C00A3F80C24B3F80C246FEA42426FEA524240
:10242C0092B2A3F80C241AE03E2E09D8720816F0CA
:10243C00010F00D00132920292B2A3F80C240EE0EC
:10244C00720916F01F0F00D1013A6FEAC2626FEAEF
:10245C00524292B2A3F80C2401E0012A2BD0B3B261
:10246C00628961692846FFF706FF6369334463613B
:10247C00236A2269934228D99B1B23626378002B21
:10248C0040D1B5F850309BB22B44227803EB0213A9
:10249C00FEB9B3F8042492B222F4F84292B2A3F833
:1024AC000424B3F804246FEA42426FEA524292B217
:1024BC00A3F8042428E0B5F8502092B22A4402EB89
:1024CC000313B2B2A3F80C24C9E7002222621E4601
:1024DC00D4E73E2E09D8720816F0010F00D0013255
:1024EC00920292B2A3F804240EE0720916F01F0FA8
:1024FC0000D1013A6FEAC2626FEA524292B2A3F87B
:10250C00042401E0012B06D0B3B22289616928466C
:10251C00FFF7B1FE3FE7B5F850309BB22B44227861
:10252C0003EB0213B2B2A3F80424EDE762788ABB82
:10253C00B5F8502092B22A4402EB03138EB9B3F8CB
:10254C00042492B222F4F84292B2A3F80424B3F811
:10255C0004246FEA42426FEA524292B2A3F8042476
:10256C001AE03E2E09D8720816F0010F00D0013285
:10257C00920292B2A3F804240EE0720916F01F0F17
:10258C0000D1013A6FEAC2626FEA524292B2A3F8EA
:10259C00042401E0012A2BD0B3B2228961692846B8
:1025AC00FFF769FE636933446361236A22699342CE
:1025BC0028D99B1B23626378002B40D1B5F850308F
:1025CC009BB22B44227803EB0213FEB9B3F80C2414
:1025DC0092B222F4F84292B2A3F80C24B3F80C2471
:1025EC006FEA42426FEA524292B2A3F80C2428E0FE
:1025FC00B5F8502092B22A4402EB0313B2B2A3F8FE
:10260C000424C9E7002222621E46D4E73E2E09D8D4
:10261C00720816F0010F00D00132920292B2A3F8A8
:10262C000C240EE0720916F01F0F00D1013A6FEA6C
:10263C00C2626FEA524292B2A3F80C2401E0012B61
:10264C0006D0B3B2628961692846FFF714FEA2E690
:10265C00B5F850309BB22B44227803EB0213B2B284
:10266C00A3F80C24EDE7217835F8212092B222F45E
:10267C00E24222F0700242F4004242F0800225F85D
:10268C002120B5F8502092B22A44217802EB011295
:10269C009BB2A2F80434228961692846FFF7EBFD4E
:1026AC0079E63E2E09D8720816F0010F00D00132DF
:1026BC00920292B2A3F80C2415E0720916F01F0FC7
:1026CC0000D1013A6FEAC2626FEA524292B2A3F8A9
:1026DC000C2408E0B5F850309BB22B4403EB0113EB
:1026EC00B2B2A3F80C246289B3B261692846FFF731
:1026FC00C2FD6378002B4CD1227835F822309BB286
:10270C0023F4E04323F0700343F4004343F0C0038D
:10271C0025F822303FE68ABBB5F850309BB22B44EB
:10272C0003EB01138EB9B3F8042492B222F4F842ED
:10273C0092B2A3F80424B3F804246FEA42426FEA7D
:10274C00524292B2A3F8042421E03E2E09D872081A
:10275C0016F0010F00D00132920292B2A3F80424B9
:10276C0015E0720916F01F0F00D1013A6FEAC26230
:10277C006FEA524292B2A3F8042408E0B5F8503044
:10278C009BB22B4403EB0113B2B2A3F804242289AD
:10279C00AAE7012B7FF4FFAD227835F822309BB2EB
:1027AC0023F4E04323F0700343F4404343F08003ED
:1027BC0025F82230EFE500228A611A467FE53E2A91
:1027CC0009D8510812F0010F00D00131890289B2E9
:1027DC00A3F80C148EE5510912F01F0F00D101392A
:1027EC006FEAC1616FEA514189B2A3F80C1481E51B
:1027FC00CB78022B45D0012B40F01D8189692369D0
:10280C00994240F2D480C91AA161D2B9B5F85020CE
:10281C0092B22A44217802EB0112002B40F0CB80BB
:10282C00B2F8041489B221F4F84189B2A2F8041464
:10283C00B2F804146FEA41416FEA514189B2A2F82F
:10284C0004146278002A40F0E880B5F8502092B267
:10285C002A44217802EB0112002B40F0C580B2F81B
:10286C000C349BB223F4F8439BB2A2F80C34B2F8AC
:10287C000C346FEA43436FEA53439BB2A2F80C3417
:10288C0038E5CAB9B0F850309BB203440A7803EB70
:10289C0002130A6972BBB3F8042492B222F4F84210
:1028AC0092B2A3F80424B3F804246FEA42426FEA0C
:1028BC00524292B2A3F804246378002B4CD1B5F8A1
:1028CC0050309BB22B44227803EB0213226952BB8B
:1028DC00B3F80C2492B222F4F84292B2A3F80C246E
:1028EC00B3F80C246FEA42426FEA524292B2A3F858
:1028FC000C2433E03E2A09D8510812F0010F00D005
:10290C0001318A0292B2A3F80424D5E7510912F0DE
:10291C001F0F00D101396FEAC1626FEA524292B2C5
:10292C00A3F80424C8E73E2A09D8510812F0010F75
:10293C0000D001318A0292B2A3F80C240EE05109A6
:10294C0012F01F0F00D101396FEAC1626FEA5242D7
:10295C0092B2A3F80C2401E0012B1DD0E369002BEB
:10296C003FF4C8AC227835F8221044F2400303EA55
:10297C0001008B4302D000287FF4BCAC35F8223028
:10298C009BB223F4E04323F0700343F4004343F081
:10299C00C00325F82230ADE4B5F850309BB22B447F
:1029AC00227803EB0213228AA3F80C24D6E7002327
:1029BC00A3610B4629E73E2B09D8590813F0010FE8
:1029CC0000D00131890289B2A2F8041439E75909FF
:1029DC0013F01F0F00D101396FEAC1616FEA514149
:1029EC0089B2A2F804142CE73E2B09D8590813F02D
:1029FC00010F00D001318B029BB2A2F80C3479E4A8
:102A0C00590913F01F0F00D101396FEAC1636FEA46
:102A1C0053439BB2A2F80C346CE4012A7FF46AACE9
:102A2C00B5F8502092B22A44217802EB01129BB2E5
:102A3C00A2F80C345EE401206DE410B45C0800EBE9
:102A4C00420000F5806007E030F8042B0A70C2F3F6
:102A5C0007224A700231013C002CF5D113F0010F12
:102A6C0001D003880B7010BC7047000008B5074AF2
:102A7C00136843F010031360032000F0B7FD00202F
:102A8C00FDF736FFFDF712FF002008BD00200240C5
:102A9C00034A1168034B1B780B441360704700BF4B
:102AAC002014002090000020014B1868704700BFD4
:102ABC002014002038B50446FFF7F6FF0546B4F1A4
:102ACC00FF3F02D0044B1B781C44FFF7EDFF401B6B
:102ADC00A042FAD338BD00BF9000002082B0084B52
:102AEC001B68084AA2FB03235B0A00FB03F3019358
:102AFC0000BF019B5A1E0192002BF9D102B0704706
:102B0C0098000020D34D6210002800F0F18170B5C0
:102B1C0082B00446036813F0010F2CD0994B5B680C
:102B2C0003F00C03042B1DD0964B5B6803F00C03D5
:102B3C00082B12D06368B3F5803F41D0002B55D1E0
:102B4C0003F1804303F504331A6822F480321A60CF
:102B5C001A6822F480221A6037E08A4B5B6813F4FF
:102B6C00803FE7D0874B1B6813F4003F03D06368AA
:102B7C00002B00F0BF81236813F0020F75D0814B3E
:102B8C005B6813F00C0F5FD07E4B5B6803F00C039B
:102B9C00082B54D02369002B00F08A807A4B012239
:102BAC001A60FFF781FF0546764B1B6813F0020F86
:102BBC0075D1FFF779FF401B0228F5D903209EE160
:102BCC00704A136843F480331360636843B3FFF7B0
:102BDC006BFF05466B4B1B6813F4003FCBD1FFF723
:102BEC0063FF401B6428F5D9032088E1B3F5A02FBF
:102BFC0009D0644B1A6822F480321A601A6822F4E5
:102C0C0080221A60E1E703F18043A3F53C331A6894
:102C1C0042F480221A601A6842F480321A60D4E7B7
:102C2C00FFF742FF0546574B1B6813F4003FA2D039
:102C3C00FFF73AFF401B6428F5D903205FE1514BA5
:102C4C005B6813F4803FA5D14E4B1B6813F0020F49
:102C5C0003D02369012B40F04F814A4A136823F0BB
:102C6C00F803616943EAC1031360236813F0080F8A
:102C7C0033D0A369002B5CD0434B0122C3F88024D2
:102C8C00FFF712FF05463F4B5B6A13F0020F21D191
:102C9C00FFF70AFF401B0228F5D903202FE1394A20
:102CAC00136823F0F803616943EAC1031360DCE79E
:102CBC00354B00221A60FFF7F7FE0546314B1B68B7
:102CCC0013F0020FD1D0FFF7EFFE401B0228F5D90D
:102CDC00032014E10120FFF701FF236813F0040F18
:102CEC0000F09680274BDB6913F0805F34D1254BC5
:102CFC00DA6942F08052DA61DB6903F080530193A8
:102D0C00019B0125214B1B6813F4807F26D0E368BF
:102D1C00012B3DD0002B53D103F1804303F5043339
:102D2C001A6A22F001021A621A6A22F004021A626A
:102D3C0033E0154B0022C3F88024FFF7B5FE05469F
:102D4C00104B5B6A13F0020FC7D0FFF7ADFE401BB0
:102D5C000228F5D90320D2E00025D3E70B4A1368EB
:102D6C0043F480731360FFF79FFE0646074B1B6806
:102D7C0013F4807FCBD1FFF797FE801B6428F5D925
:102D8C000320BCE0001002400000424200700040F2
:102D9C005F4A136A43F001031362E36833B3FFF72E
:102DAC0083FE06465A4B1B6A13F0020F2FD1FFF716
:102DBC007BFE801B41F288339842F3D903209EE0BE
:102DCC00052B09D0524B1A6A22F001021A621A6AB8
:102DDC0022F004021A62E0E74D4B1A6A42F0040238
:102DEC001A621A6A42F001021A62D6E7FFF75CFE19
:102DFC000646474B1B6A13F0020F08D0FFF754FE30
:102E0C00801B41F288339842F3D9032077E0E5B96F
:102E1C00E369002B72D03E4A526802F00C02082A79
:102E2C0056D0022B17D03B4B00221A66FFF73CFE04
:102E3C000446374B1B6813F0007F47D0FFF734FE76
:102E4C00001B0228F5D9032059E0314AD36923F03D
:102E5C008053D361DCE72F4B00221A66FFF724FE68
:102E6C0005462B4B1B6813F0007F06D0FFF71CFEAA
:102E7C00401B0228F5D9032041E0236AB3F5803FBB
:102E8C001AD023494B6823F47413226A606A0243F4
:102E9C0013434B601F4B01221A66FFF705FE0446D5
:102EAC001B4B1B6813F0007F0ED1FFF7FDFD001BC1
:102EBC000228F5D9032022E0154A536823F4003385
:102ECC00A1680B435360DCE7002018E0002016E0FB
:102EDC00012B16D00E4B5B6803F48031226A9142B1
:102EEC0011D103F47013626A93420ED1002006E0F4
:102EFC0001207047012002E0012000E0002002B018
:102F0C0070BD0120FBE70120F9E70120F7E700BFC6
:102F1C000010024000004242014B0122DA6470476B
:102F2C000000424286B0174B0FCB0DF1180C0CE988
:102F3C000F0040F20123ADF80430134B5B6803F033
:102F4C000C02082A02D0114806B07047C3F3834222
:102F5C0018326A4412F8100C13F4803F0DD00A4B4F
:102F6C005B68C3F3404318336B4413F8143C074AB3
:102F7C0002FB00F0B0FBF3F0E6E7054B03FB00F0BF
:102F8C00E2E700BF445200080010024000127A0031
:102F9C0000093D00002800F0A08070B50D460446E5
:102FAC00524B1B6803F007038B420BD24F4A13683A
:102FBC0023F007030B431360136803F007038B42E2
:102FCC0040F08D80236813F0020F17D013F0040F1C
:102FDC0004D0474A536843F4E0635360236813F00A
:102FEC00080F04D0424A536843F460535360404A7C
:102FFC00536823F0F003A1680B435360236813F06C
:10300C00010F31D06368012B20D0022B25D0384A18
:10301C00126812F0020F64D035494A6822F003029C
:10302C0013434B60FFF740FD0646314B5B6803F0E2
:10303C000C036268B3EB820F16D0FFF735FD801BD3
:10304C0041F288339842F0D9032045E0284A1268AF
:10305C0012F4003FE0D101203EE0254A126812F044
:10306C00007FD9D1012037E0204B1B6803F0070308
:10307C00AB420AD91D4A136823F007032B43136094
:10308C00136803F00703AB422DD1236813F0040F30
:10309C0006D0174A536823F4E063E1680B4353608E
:1030AC00236813F0080F07D0114A536823F46053B8
:1030BC00216943EAC1035360FFF734FF0C4B5B6893
:1030CC00C3F303130B4AD35CD8400B4B18600B4B68
:1030DC001868FDF70DFC002070BD01207047012021
:1030EC00FAE70120F8E70120F6E700BF00200240D4
:1030FC000010024058520008980000209400002054
:10310C00014B1868704700BF9800002008B5FFF706
:10311C00F7FF044B5B68C3F30223034AD35CD8402C
:10312C0008BD00BF00100240685200080F23036066
:10313C000B4B5A6802F0030242605A6802F0F0022C
:10314C0082605A6802F4E062C2605B68DB0803F4D8
:10315C00E0630361034B1B6803F007030B607047CC
:10316C0000100240002002407047000008B5064BDA
:10317C009B6813F0800F00D108BDFFF7F5FF024BE1
:10318C0080229A72F8E700BF0010024070B582B03E
:10319C000446036813F0010F36D03F4BDB6913F084
:1031AC00805F49D13C4BDA6942F08052DA61DB69CD
:1031BC0003F080530193019B0125384B1B6813F4DA
:1031CC00807F3BD0344B1B6A13F4407313D062687E
:1031DC0002F440729A420ED02F4A136A23F44070C4
:1031EC002F490126C1F840640026C1F840641062E2
:1031FC0013F0010F36D1284A136A23F44073616827
:10320C000B431362002D3ED1236813F0020F06D03E
:10321C00214A536823F44043A1680B43536023684D
:10322C0013F0100F34D01C4A536823F48003E16868
:10323C000B43536000202CE00025BEE7174A1368AF
:10324C0043F480731360FFF72FFC0646134B1B6887
:10325C0013F4807FB6D1FFF727FC801B6428F5D9C7
:10326C00032016E0FFF720FC06460B4B1B6A13F0FD
:10327C00020FC0D1FFF718FC801B41F28833984233
:10328C00F3D9032005E0D36923F08053D361BBE766
:10329C00002002B070BD00BF001002400070004062
:1032AC000000424270B582B00024A446A6E0804DD6
:1032BC00AB4210D007D97F4DAB420CD005F5803511
:1032CC00AB4208D013E0A5F58015AB4203D005F551
:1032DC007025AB4207D18B68002B58D0012B51D0F5
:1032EC004261082403E0A5F58015AB42F3D0BEF192
:1032FC00FF0F4ED80646BEF1FF0F4CD84FEA8C029A
:10330C0033680F25954023EA050304FA02F21343B0
:10331C0033604B6813F0805F6ED0674B9A6942F054
:10332C0001029A619B6903F001030193019B4FEA2F
:10333C009C02951C614B53F825600CF00305AD0005
:10334C000F23AB4026EA03065D4B984229D003F5C8
:10335C008063984200F08E8003F58063984200F001
:10336C008B8003F58063984219D004231AE0CC6853
:10337C00BDE7CC680434BAE7CC680834B7E7CC684E
:10338C000C34B4E702610824B1E70024AFE704244D
:10339C00ADE7061DAFE7ACF108029200B0E70323DE
:1033AC0000E00023AB4033430232444D45F8223059
:1033BC004B6813F4803F61D0424A136843EA0E0312
:1033CC0013604B6813F4003F5ED03E4A536843EAE7
:1033DC000E0353604B6813F4801F5BD0394A93681B
:1033EC0043EA0E0393604B6813F4001F58D0354A20
:1033FC00D36843EA0E03D3600CF1010C0B6833FA6B
:10340C000CF253D0012202FA0CF203EA020E32EA59
:10341C000303F1D14B68122B3FF649AF122B3FF649
:10342C0066AF01A555F823F0E33200087B330008A2
:10343C008533000897330008FB320008FB32000884
:10344C00FB320008FB320008FB320008FB3200089C
:10345C00FB320008FB320008FB320008FB3200088C
:10346C00FB320008FB320008FB3200087F330008F7
:10347C008B330008012395E7022393E7114A136865
:10348C0023EA0E0313609CE70E4A536823EA0E03EB
:10349C0053609FE70B4A936823EA0E039360A2E7FD
:1034AC00084AD36823EA0E03D360A5E702B070BDC7
:1034BC0000002210000031100010024000000140FA
:1034CC00000801400004014000226EE0032500E0EA
:1034DC00002505FA04F4644544D0FF2B5CD88646DD
:1034EC00FF2B5CD89500DEF800404FF00F0C0CFA67
:1034FC0005FC24EA0C044FF0040C0CFA05FC44EA1D
:10350C000C04CEF80040C46824EA0303C360013203
:10351C0031FA02F347D0012393400B40F7D09608C1
:10352C00B51C274C54F8255002F00304A4004FF0AE
:10353C000F0C0CFA04FE0EEA050C224DA842C7D063
:10354C0005F58065A84209D005F58065A84207D02D
:10355C0005F58065A842B9D00425BAE70125B8E77E
:10356C000225B6E7164FB41C57F8245025EA0E0571
:10357C0047F82450144C256825EA03052560656836
:10358C0025EA03056560A56825EA0305A560E568DD
:10359C0025EA0305E560A0E700F1040EA0E7A2F11F
:1035AC000805AD009FE7F0BD013231FA02F305D0FA
:1035BC00012393400B40F7D0F0B5B0E7704700BF44
:1035CC000000014000080140000401400AB1016103
:1035DC007047090401617047C36801EA030221EADC
:1035EC00030141EA0241016170470000074AD368B8
:1035FC0023F4E0631B041B0C000200F4E0600343A3
:10360C0043F0BF6343F40033D360704700ED00E038
:10361C0000B5194BDB68C3F30223C3F1070CBCF1F3
:10362C00040F28BF4FF0040C03F1040EBEF1060F7B
:10363C0018D9033B4FF0FF3E0EFA0CFC21EA0C01AB
:10364C0099400EFA03FE22EA0E020A4300280BDB15
:10365C001201D2B200F1604000F5614080F8002305
:10366C005DF804FB0023E5E700F00F001201D2B275
:10367C00024B1A54F4E700BF00ED00E014ED00E03B
:10368C00002807DB00F01F02400901239340024A87
:10369C0042F82030704700BF00E100E070470000A6
:1036AC0090F83D30DBB2012B27D1022380F83D305E
:1036BC000268D36843F00103D3600368114A934254
:1036CC0010D0B3F1804F0DD0A2F59432934209D0B3
:1036DC0002F58062934205D01A6842F001021A602A
:1036EC00002070479A6802F00702062A07D01A6871
:1036FC0042F001021A600020704701207047002040
:10370C00704700BF002C01407047704770477047EE
:10371C0010B5044603681A6912F0020F11D0DA686A
:10372C0012F0020F0DD06FF002021A610123037721
:10373C0003689B6913F0030F70D0FFF7E6FF0023BB
:10374C00237723681A6912F0040F12D0DA6812F08A
:10375C00040F0ED06FF004021A6102232377236842
:10376C009B6913F4407F5FD02046FFF7CEFF002308
:10377C00237723681A6912F0080F12D0DA6812F056
:10378C00080F0ED06FF008021A6104232377236808
:10379C00DB6913F0030F4ED02046FFF7B6FF002372
:1037AC00237723681A6912F0100F12D0DA6812F01E
:1037BC00100F0ED06FF010021A61082323772368C4
:1037CC00DB6913F4407F3DD02046FFF79EFF0023BA
:1037DC00237723681A6912F0010F03D0DA6812F00C
:1037EC00010F36D123681A6912F0800F03D0DA6802
:1037FC0012F0800F34D123681A6912F0400F03D0F5
:10380C00DA6812F0400F32D123681A6912F0200FD7
:10381C0003D0DA6812F0200F30D110BDFFF774FF1F
:10382C002046FFF773FF8AE72046FFF76DFF20461F
:10383C00FFF76CFF9BE72046FFF766FF2046FFF77C
:10384C0065FFACE72046FFF75FFF2046FFF75EFF02
:10385C00BDE76FF001021A612046FCF731FFC1E7AA
:10386C006FF080021A61204600F077F8C3E76FF022
:10387C0040021A612046FFF74AFFC5E76FF02002AD
:10388C001A61204600F068F8C7E7000003681B4A7D
:10389C0090420AD0B0F1804F07D0A2F594329042FA
:1038AC0003D002F58062904203D123F070034A6882
:1038BC001343124A90420AD0B0F1804F07D0A2F5C0
:1038CC009432904203D002F58062904203D123F4EB
:1038DC004073CA68134323F080034A69134303609F
:1038EC008B68C3620B688362044B984202D001233D
:1038FC00436170470B690363F9E700BF002C01407B
:10390C0040B310B5044690F83D30F3B1022384F86F
:10391C003D30214651F8040BFFF7B8FF012384F822
:10392C00463084F83E3084F83F3084F8403084F8D8
:10393C00413084F8423084F8433084F8443084F8C1
:10394C00453084F83D30002010BD80F83C30FFF746
:10395C00A5FEDBE70120704770477047034B5B689F
:10396C00C3F30313024AD35CD840704700100240E3
:10397C0058520008034B5B68C3F30223024AD35C22
:10398C00D84070470010024068520008034B5B6837
:10399C00C3F3C223024AD35CD840704700100240E4
:1039AC00685200080B4B5B6803F4803343B90A4838
:1039BC00084B5B68C3F38343023303FB00F070478F
:1039CC00044B5B68C3F3404301330448B0FBF3F092
:1039DC00EEE700BF0010024000093D0000127A0023
:1039EC0008B5054B5B6803F00C03082B01D00348AA
:1039FC0008BDFFF7D7FFFBE70010024000127A006A
:103A0C0010B50446FFF7ECFF2060FFF7A7FF6060DE
:103A1C00FFF7B0FFA0606068FFF7B8FFE06010BD73
:103A2C00704798B108B50346D0F8B40210B1002025
:103A3C00C3F8B40209B1C3F8B012012183F89C1287
:103A4C001A701846FDF70AF9002008BD02207047CD
:103A5C0019B1C0F8B412002070470220704708B5A5
:103A6C00FDF73EF9002008BD08B5D0F8B4322BB1F3
:103A7C001B68984700B908BD0220FCE70220FAE752
:103A8C0008B5D0F8B4325B689847002008BD38B54B
:103A9C00044600F52A75284600F035F90123C4F8D0
:103AAC009432B4F8AE32C4F8983294F8A81201F0FB
:103ABC001F03012B0ED0022B11D02BB101F0800172
:103ACC002046FDF728F903E02946204600F0CAFA03
:103ADC00002038BD2946204600F0F8FAF8E72946C0
:103AEC00204600F023FBF3E738B504460D4691BBA6
:103AFC001346D0F89422032A03D0052A24D0084672
:103B0C0033E0D0F86011D0F8642191420DD9891AB4
:103B1C00C0F860118A4206D98AB21946204600F0D4
:103B2C0037FC284621E092B2F7E7D0F8B4321B6993
:103B3C001BB190F89C22032A04D0204600F030FCE4
:103B4C00284612E09847F8E70021C0F89412FDF7D8
:103B5C00E2F8284609E0D0F8B4329B6933B190F80A
:103B6C009C22032A04D19847002038BD0220FCE790
:103B7C000220FAE738B504460D46002953D1134606
:103B8C00D0F89422022A0CD0042A00D01AB9802131
:103B9C002046FDF7C0F894F8A032012B3ED0284601
:103BAC0038BD026A416A8A421BD8C269B2FBF1F382
:103BBC0001FB13232BB9914203D8D0F898329A42C7
:103BCC001CD3D4F8B432DB681BB194F89C22032AC2
:103BDC0021D080212046FDF79EF8204600F0EBFB1B
:103BEC00D9E7521A026292B2194600F0BAFB0023CE
:103BFC001A4619462046FDF7C5F8CCE700221146B7
:103C0C0000F0AFFB0021C4F898120B460A46204680
:103C1C00FDF7B8F8BFE720469847DAE7002384F8A9
:103C2C00A0322846BCE7D0F8B4325B6933B190F8C7
:103C3C009C22032A04D198470020B1E70220AFE769
:103C4C000220ADE770B50446402300221146FDF773
:103C5C004FF80125C4F858514026C4F86461334626
:103C6C00002280212046FDF743F8A561666284F8A6
:103C7C009C520023C4F894326360C4F8A432D4F884
:103C8C00B8322BB1D4F8B4325B6800212046984787
:103C9C00002070BD01740020704790F89C3280F8B1
:103CAC009D32042380F89C320020704790F89C329F
:103CBC00042B01D00020704790F89D3280F89C3284
:103CCC00F8E708B590F89C32032B01D0002008BD12
:103CDC00D0F8B432DB69002BF8D09847F6E70346EE
:103CEC00002002E00130C0B201331A78002AF9D169
:103CFC00704708B54B88012B00D008BDC0F8A43222
:103D0C0000F04EFBF9E70B7803704B7843708B781F
:103D1C00CA7803EB022343800B794A7903EB022325
:103D2C0083808B79CA7903EB0223C380704710B56B
:103D3C0004468021FCF7EFFF00212046FCF7EBFF47
:103D4C0010BD30B583B005460C460023ADF80630E7
:103D5C004A88130A013B062B00F2A480DFE803F02B
:103D6C0004182CA2A2869300D0F8B0321B680DF177
:103D7C000601007C9847BDF806201AB1E388002B99
:103D8C0040F09480E388002B00F09A8003B030BDA3
:103D9C00037C43B9D0F8B4329B6A0DF10600984706
:103DAC0002234370E7E7D0F8B432DB6A0DF106006A
:103DBC00984702234370DEE7D2B2052A52D8DFE8D7
:103DCC0002F003101D2A3744D0F8B0325B6823B1DF
:103DDC000DF10601007C9847CDE72146FFF7A7FFC0
:103DEC00D4E7D0F8B0329B6823B10DF10601007C0A
:103DFC009847C0E72146FFF79AFFC7E7D0F8B032E3
:103E0C00DB6823B10DF10601007C9847B3E721462E
:103E1C00FFF78DFFBAE7D0F8B0321B6923B10DF173
:103E2C000601007C9847A6E72146FFF780FFADE727
:103E3C00D0F8B0325B6923B10DF10601007C9847D4
:103E4C0099E72146FFF773FFA0E7D0F8B0329B69E2
:103E5C0023B10DF10601007C98478CE72146FFF752
:103E6C0066FF93E72146FFF762FF8FE7037C33B9C8
:103E7C00D0F8B4325B6B0DF1060098477BE7214616
:103E8C00FFF755FF82E7037C43B9D0F8B4321B6BC4
:103E9C000DF106009847072343706CE72146FFF7A6
:103EAC0046FF73E72146FFF742FF6FE79A4228BFB0
:103EBC001A46ADF806200146284600F045FA61E79F
:103ECC00284600F06DFA61E738B504468B88F3B9E3
:103EDC00CB88E3B94B887F2B19D803F07F0590F87A
:103EEC009C32032B0CD080F89E522946FCF73AFFEB
:103EFC00204600F055FA35B1022384F89C3209E0D3
:103F0C00FFF715FF06E0012384F89C3202E02046FF
:103F1C00FFF70DFF38BD000038B504460D46897813
:103F2C00284B197001290ED890F89C32022B0ED018
:103F3C00032B21D02946FFF7FAFE224B1978204695
:103F4C00FFF79EFD02E02946FFF7F1FE38BD81B177
:103F5C004160032380F89C32FFF786FD022803D0D2
:103F6C00204600F01DFAF1E729462046FFF7DFFE58
:103F7C00ECE700F015FAE9E789B1436899421DD0E6
:103F8C00D9B2FFF77DFD0F4B197861602046FFF722
:103F9C006BFD02280DD0204600F002FAD6E7022372
:103FAC0080F89C324160FFF76BFD204600F0F8F979
:103FBC00CCE729462046FFF7BAFEC7E700F0F0F938
:103FCC00C4E700BF2414002008B5CB88012B0AD10C
:103FDC0090F89C32022B09D9032B09D10122011D27
:103FEC0000F0B2F901E0FFF7A2FE08BD5BB213B915
:103FFC00FFF79DFEF9E70146002341F8083F012237
:10400C0000F0A2F9F1E708B590F89C32013B022BC5
:10401C0012D8CB88022B0CD10123C360D0F8A43268
:10402C000BB10323C360022200F10C0100F08CF9E8
:10403C0008BDFFF77CFEFBE7FFF779FEF8E708B554
:10404C0090F89C32013B022B09D84B88012B00D0F5
:10405C0008BD0023C0F8A43200F0A2F9F8E7FFF77E
:10406C0066FEF5E708B50B7803F06003202B05D04E
:10407C00402B03D043B1FFF75AFE03E0D0F8B43223
:10408C009B689847002008BD4B78092B1BD8DFE8AC
:10409C0003F011171A141A08051A0E0BFFF751FE2C
:1040AC00F0E7FFF711FFEDE7FFF736FFEAE7FFF761
:1040BC008BFFE7E7FFF7A7FFE4E7FFF71AFEE1E75F
:1040CC00FFF7BDFFDEE7FFF732FEDBE738B505464D
:1040DC000C460B7803F06003202B06D0402B04D049
:1040EC001BB1FFF724FE002038BD95F89C32013B34
:1040FC00022B16D82379012B0ED8D5F8B4329B6835
:10410C00214628469847E388002BECD10028EAD1B9
:10411C00284600F045F9E6E721462846FFF707FE5A
:10412C00E1E721462846FFF702FEDCE770B50546BD
:10413C008B880C7804F06004202C07D0DAB2402C69
:10414C0004D05CB1FFF7F3FD002405E0D5F8B432E0
:10415C009B68284698470024204670BD202C09D027
:10416C004E78012E33D0032E0AD0002E55D0FFF7F7
:10417C00DEFDF1E7D0F8B4329B6898470446EBE7D4
:10418C0090F89C32022B04D0032B11D0FFF7CFFDFB
:10419C00E2E70AB1802A03D12846FFF7C8FDDBE726
:1041AC001146FCF7B8FD80212846FCF7B4FDD3E797
:1041BC004B8823B91AB1802A01D0CB881BB1284671
:1041CC0000F0EEF8C8E71146FCF7A5FDF7E790F80C
:1041DC009C32022B04D0032B11D0FFF7A8FDBBE7B8
:1041EC000AB1802A03D12846FFF7A1FDB4E7114696
:1041FC00FCF791FD80212846FCF78DFDACE74B8840
:10420C00002BA9D112F07F0F03D1284600F0C8F87B
:10421C00A2E71146FCF787FDF7E790F89C0202280D
:10422C0006D0032829D02846FFF781FD344693E7B2
:10423C000AB1802A13D113F0800F15D102F07F023E
:10424C0002EB8202910001F5A8712944043100238C
:10425C000B600222284600F077F834467CE72846AB
:10426C00FFF765FD344677E702F07F0202EB82022E
:10427C009100103129440431E9E75BB2002B1FDBBC
:10428C0002F00F0000EB800005EB8000D0F8580125
:10429C0020B3002B27DB02F07F0303EB83039C008E
:1042AC0004F5A8742C4404340AB1802A24D10023C8
:1042BC00236002222146284600F046F834464BE79C
:1042CC0002F00F0000EB800005EB800080690028F5
:1042DC00DFD12846FFF72BFD34463DE72846FFF794
:1042EC0026FD344638E702F07F0303EB83039C0082
:1042FC0010342C440434D7E711462846FCF71BFD38
:10430C0010B101232360D4E700232360D1E7D0B19F
:10431C0070B50D4616460446FFF7E1FC431C5B00E6
:10432C009BB233802B7003236B70022307E00134A4
:10433C005A1CD2B2E8540233DBB20021A9542078C3
:10434C000028F4D170BD704708B513460222C0F89E
:10435C009422C36103620A460021FCF70BFD002086
:10436C0008BD08B513460A460021FCF703FD0020E2
:10437C0008BD08B513460322C0F89422C0F85C317E
:10438C00C0F860310A460021FCF7FCFC002008BD97
:10439C0008B513460A460021FCF7F4FC002008BDC2
:1043AC0008B50423C0F8943200231A461946FCF7CA
:1043BC00E1FC002008BD08B50523C0F894320023A9
:1043CC001A461946FCF7DEFC002008BD10B5D0F8E3
:1043DC00B842D0F8BC325BB194F80002FF2807D089
:1043EC009B6894F8012221469847FF2384F80032F9
:1043FC00002010BD4323038000487047D4000020E8
:10440C004323038000487047180100204323038096
:10441C0000487047680100200A2303800048704759
:10442C005C01002038B50446D0F8B852FCF7B2FC59
:10443C00C5F80C02D4F8B8324BB1D4F8BC32DB68F6
:10444C0005F50371D5F804029847002038BD022009
:10445C00FCE710B5D0F8B822D0F8C042F2B101EBAD
:10446C00810300EB8303DB694BB101EB810C04EBA3
:10447C00CC04A46BB3FBF4FC04FB1C3323B100236E
:10448C00C2F81432002010BD01EB810300EB830352
:10449C000022DA611346FCF76DFCF3E70220F2E729
:1044AC00F0B583B006460C46D0F8B87200238DF8F0
:1044BC000730ADF804300B7813F0600527D0202DB1
:1044CC0053D1CA88DAB113F0800F0CD0D0F8BC32BB
:1044DC009B68394660789847E28839463046FFF742
:1044EC0033FF002544E04B7887F800328B7987F84E
:1044FC000132CA883946FFF73CFF002538E0D0F876
:10450C00BC329B68002248789847002530E04F78F1
:10451C000A2F14D00B2F20D01FB1FFF708FC022557
:10452C0026E090F89C32032B03D0FFF700FC022509
:10453C001EE0022201A9FFF707FF3D4618E090F8A4
:10454C009C32032B03D0FFF7F2FB022510E0012273
:10455C000DF10701FFF7F8FE0AE090F89C32032BEF
:10456C0006D0FFF7E4FB022502E0FFF7E0FB022593
:10457C00284603B0F0BD38B504468121FCF7C3FBD7
:10458C000025E56201212046FCF7BDFBC4F86C5107
:10459C0082212046FCF7B7FB2564D4F8B8324BB126
:1045AC00D4F8BC325B689847D4F8B802FCF7FCFB33
:1045BC00C4F8B852002038BD70B50446037CABBBC0
:1045CC004FF4007302228121FCF792FB0125E56276
:1045DC004FF40073022229462046FCF789FBC4F8ED
:1045EC006C510823032282212046FCF781FB012316
:1045FC0023644FF40770FCF7D3FB0546C4F8B802EC
:10460C0068B3D4F8BC321B6898470023C5F8143241
:10461C00C5F81832267CCEB94FF40073D5F80422B5
:10462C0001212046FCF7AEFB304670BD4023022230
:10463C008121FCF75DFB0125E5624023022229461E
:10464C002046FCF755FBC4F86C51CAE74023D5F85B
:10465C00042201212046FCF795FB0026E4E7012605
:10466C00E2E719B1C0F8BC12002070470220704775
:10467C00D0F8B832C3F80812C3F8102200207047E3
:10468C00D0F8B832C3F8041200207047D0F8B82222
:10469C00A2B108B5D2F814320BB1012008BD012328
:1046AC00C2F81432D2F810320363B2F81032D2F8D6
:1046BC0008228121FCF75EFB0020EFE70220704707
:1046CC00D0F8B82292B108B5037C43B94FF400730B
:1046DC00D2F804220121FCF755FB002008BD402331
:1046EC00D2F804220121FCF74DFBF6E702207047BB
:1046FC0008B338B5044603684CF6CC421A6003681C
:10470C0045F255521A60036842685A600368826821
:10471C009A60FEF7C9F905462368DA6832B1FEF7EC
:10472C00C3F9401B2628F7D9032003E04AF6AA2236
:10473C001A60002038BD0120704703684AF6AA228F
:10474C001A60002070470000002103E00B4B5B58FF
:10475C00435004310A480B4B42189A42F6D30A4A8A
:10476C0002E0002342F8043B084B9A42F9D3FFF7CE
:10477C0057F900F00FF8FCF70BF87047AC52000833
:10478C00000000201002002010020020381400202D
:10479C00FEE7000070B500260C4D0D4C641BA410F8
:1047AC00A64209D100F084FC00260A4D0A4C641B79
:1047BC00A410A64205D170BD55F8043B98470136AC
:1047CC00EEE755F8043B98470136F2E7A45200088F
:1047DC00A4520008A4520008A85200080346024440
:1047EC00934200D1704703F8011BF9E70CB430B5C4
:1047FC00174B0C1E1D689DB008DA8B234FF0FF3051
:10480C002B601DB0BDE8304002B070474FF402730E
:10481C00ADF814300CBF234604F1FF330493079317
:10482C004FF6FF7302900690ADF81630284621AB78
:10483C00209A02A9019300F06BF8431CBCBF8B2398
:10484C002B60002CDDD00022029B1A70D9E700BF30
:10485C00AC010020704770472DE9F0478E68824606
:10486C009E420C4690461F4638D88A8912F4906FA7
:10487C0032D0256809690133A5EB010965694B4400
:10488C0005EB450505EBD5756D109D4238BF1D46F2
:10489C00530531D5294600F04FFB064650B90C2381
:1048AC004FF0FF30CAF80030A38943F04003A381D6
:1048BC00BDE8F0874A46216900F0CEFAA38923F4BB
:1048CC00906343F08003A38126614E4426603E46EC
:1048DC006561A5EB0905A560BE4200D93E4632468E
:1048EC004146206800F0C6FAA36800209B1BA36019
:1048FC00236833442360DBE72A4600F077FB064647
:10490C000028E1D15046216900F0CEFAC7E700003B
:10491C002DE9F04F98468B8907461B060D46144629
:10492C009DB00ED50B6963B9402100F005FB2860E2
:10493C00286120B90C233B604FF0FF30D1E04023BD
:10494C006B610023099320238DF8293030234FF01D
:10495C000109CDF80C80DFF8A4818DF82A302346AC
:10496C009A4613F8012B0AB1252AF9D1BAEB040B9C
:10497C000BD05B46224629463846FFF76DFF0130C7
:10498C0000F0AA80099A5A4409929AF80030002B38
:10499C0000F0A28000234FF0FF32CDE905230AF18D
:1049AC00010A049307938DF853301A935446052249
:1049BC0014F8011B514800F041FA049AD8B9D006FA
:1049CC0044BF20238DF85330110744BF2B238DF89F
:1049DC0053309AF800302A2B15D0544600204FF053
:1049EC000A0C079A214611F8013B303B092B4ED992
:1049FC00B0B1079214E0A0EB080309FA03F31343D8
:104A0C00A2460493D2E7039B191D1B680391002B4C
:104A1C00BBBF5B4242F0020207930793B8BF0492FC
:104A2C0023782E2B0CD163782A2B35D1039B02349F
:104A3C001A1D1B680392002BB8BF4FF0FF33059370
:104A4C00DFF8BCA003225046217800F0F7F940B102
:104A5C004023A0EB0A0003FA00F0049B013403434B
:104A6C00049314F8011B062226488DF8281000F038
:104A7C00E5F9002838D0244B1BBB039B073323F0EC
:104A8C00070308330393099B3344099367E70C46E8
:104A9C0001200CFB0232A5E700234FF00A0C19464B
:104AAC0001340593204610F8012B303A092A03D91A
:104ABC00002BC5D00591C3E7044601230CFB012153
:104ACC00F0E703AB00932A463846104B04A9AFF32A
:104ADC000080421C0646D6D1AB895B063FF52CAF55
:104AEC0009981DB0BDE8F08F03AB00932A463846F9
:104AFC00064B04A900F07CF8EBE700BF70520008ED
:104B0C00765200087A520008000000006548000840
:104B1C002DE9F047164699468A680B690746934279
:104B2C00B8BF1346336091F843200C46DDF8208063
:104B3C000AB1013333602368990642BF33680233EC
:104B4C003360256815F0060506D104F1190AE368EF
:104B5C0032689B1AAB4228DC94F84320131E22685F
:104B6C0018BF012392062DD44946384604F143025E
:104B7C00C047013020D02368E56803F00603042BFE
:104B8C0018BF002532684FF00006A36808BFAD1AA5
:104B9C00226908BF25EAE5759342C4BF9B1AED183C
:104BAC001A34B5421AD1002008E001235246494676
:104BBC003846C047013003D14FF0FF30BDE8F087D5
:104BCC000135C4E73020E11881F843005A1C94F8F1
:104BDC0045102244023382F84310C5E701232246D4
:104BEC0049463846C0470130E6D00136D9E70000C7
:104BFC002DE9FF470F7E9146782F80460C469A464A
:104C0C000C9D01F1430207D8622F0AD8002F00F047
:104C1C00D980582F00F0A48004F1420584F842702A
:104C2C003AE0A7F16303152BF6D801A151F823F054
:104C3C00954C0008A94C0008254C0008254C000890
:104C4C00254C0008254C0008A94C0008254C0008F0
:104C5C00254C0008254C0008254C0008B74D0008D1
:104C6C00D94C0008994D0008254C0008254C00082B
:104C7C00D94D0008254C0008D94C0008254C0008DB
:104C8C00254C0008A14D00082B681A1D1B682A60D2
:104C9C0004F1420584F842300123A4E0206829681D
:104CAC00060601F104030AD50E682B60002E03DA08
:104CBC002D23764284F843300A235E4819E00E68AF
:104CCC0010F0400F2B6018BF36B2EFE72B6820684E
:104CDC00191D2960010601D51E6802E04606FBD5A8
:104CEC001E886F2F0CBF08230A235248002184F81A
:104CFC0043106568002DA8BF2168A560A4BF21F0F2
:104D0C00040121600EB9002D4DD01546B6FBF3F110
:104D1C0003FB1167C75D05F8017D3746BB420E46A4
:104D2C00F4D9082B0BD12368DE0708D523696168F9
:104D3C009942DEBF302305F8013C05F1FF35521BCB
:104D4C0022614B4621464046CDF800A003AAFFF74E
:104D5C00DFFE01304CD14FF0FF3004B0BDE8F087DE
:104D6C00344881F845702968236851F8046B296030
:104D7C001D0614D5DF0744BF43F0200323601EB982
:104D8C00236823F0200323601023AFE7236843F04C
:104D9C00200323607823284884F84530E3E759063C
:104DAC0048BFB6B2E6E71546BBE72B682668181D68
:104DBC006169286035061B6801D5196002E0700630
:104DCC00FBD51980002315462361BAE72B68002117
:104DDC001A1D2A601D686268284600F02FF808B179
:104DEC00401B606063682361002384F84330A8E7AC
:104DFC002A46494640462369D0470130ABD0236848
:104E0C009B0713D4E068039B9842B8BF1846A4E7ED
:104E1C000123324649464046D04701309BD00135EC
:104E2C00E36803995B1AAB42F2DCEBE7002504F173
:104E3C001906F5E78152000892520008034610B596
:104E4C00C9B202449342184601D1002003E0047811
:104E5C0001338C42F6D110BD0A44914200F1FF336C
:104E6C0000D1704710B511F8014B914203F8014F76
:104E7C00F9D110BD884210B501EB020402D984426D
:104E8C00234607D8431EA14208D011F8012B03F882
:104E9C00012FF8E7014602448A4200D110BD13F8F5
:104EAC00014D02F8014DF7E738B50546002940D011
:104EBC0051F8043C0C1F002BB8BFE41800F0D6F8D6
:104ECC001C4A136833B9636014602846BDE8384047
:104EDC0000F0D2B8A34208D9206821188B4201BF38
:104EEC0019685B6809182160EDE71A465B680BB11D
:104EFC00A342FAD911685018A0420BD12068014482
:104F0C00501883421160E0D118685B68014411604D
:104F1C005360DAE702D90C232B60D6E720682118FE
:104F2C008B4201BF19685B6809182160636054608B
:104F3C00CBE738BD28140020F8B5CD1C25F00305AF
:104F4C0008350C2D38BF0C25002D064601DBA94277
:104F5C0003D90C2333600020F8BD00F087F82149F9
:104F6C000A6814469CB9204F3B6823B92146304649
:104F7C0000F06CF838602946304600F067F8431CA6
:104F8C0023D10C233046336000F076F8E3E7236836
:104F9C005B1B17D40B2B03D923601C44256004E046
:104FAC006368A2420CBF0B605360304600F064F89B
:104FBC0004F10B00231D20F00700C21ACCD01B1AE1
:104FCC00A350C9E722466468CCE7C41C24F0030450
:104FDC00A042E3D0211A304600F038F80130DDD180
:104FEC00CFE700BF281400202C1400202DE9F0413D
:104FFC00804614460E4621B91146BDE8F041FFF734
:10500C009BBF2AB9FFF750FF25462846BDE8F08123
:10501C0000F038F88442074602D8B4EB500F12D88F
:10502C0021464046FFF788FF05460028EDD0BC42DC
:10503C002246314628BF3A46FFF70EFF314640461E
:10504C00FFF732FFE1E73546DFE7000038B5002314
:10505C00054D044608462B6000F01CF8431C02D199
:10506C002B6803B1236038BD301400200148FFF7D2
:10507C00F1BB00BF251400200148FFF7ECBB00BFBB
:10508C002514002051F8043C181F002BBCBF0B58F2
:10509C00C0187047044A05491368002B08BF0B461B
:1050AC00184410601846704734140020381400203F
:1050BC00F8B500BFF8BC08BC9E467047F8B500BFF9
:0850CC00F8BC08BC9E467047C9
:1050D400005EBCE2613FDD83C29C7E20A3FD1F41D4
:1050E4009DC3217FFCA2401E5F01E3BD3E6082DCC4
:1050F400237D9FC1421CFEA0E1BF5D0380DE3C62B4
:10510400BEE0025CDF81633D7C22C09E1D43A1FFA3
:105114004618FAA427799BC584DA3866E5BB590793
:10512400DB856739BAE406581947A5FB7826C49A83
:10513400653BD987045AB8E6A7F91B45C6987A2473
:10514400F8A6441A99C7257B3A6486D85B05E7B963
:105154008CD2306EEDB3510F4E10F2AC2F7193CD53
:10516400114FADF3702ECC92D38D6F31B2EC0E5043
:10517400AFF1134DCE90722C6D33D18F0C52B0EE33
:10518400326C8ED0530DEFB1F0AE4C1291CF2D7323
:10519400CA947628ABF517490856B4EA6937D58B13
:1051A4005709EBB536688AD495CB2977F4AA481603
:1051B400E9B7550B88D6346A2B7597C94A14F6A8F3
:1051C400742AC896154BA9F7B6E80A54D7896B35E3
:1051D40025303278253032782530327825303278CF
:1051E40025303278253032782530327825303278BF
:1051F4000925640D0A00000053544D3332205669CA
:10520400727475616C20436F6D506F72740000008E
:1052140053544D6963726F656C656374726F6E6924
:105224006373000043444320436F6E666967000064
:1052340043444320496E74657266616365000000EF
:1052440002030405060708090A0B0C0D0E0F1010C3
:105254000000000000000000000000000102030440
:10526400060708090000000001020304232D302B67
:105274002000686C4C006566674546470030313253
:1052840033343536373839414243444546003031AA
:105294003233343536373839616263646566000009
:0452A40041010008BC
:0452A8001D010008DC
:1052AC00280000206D040008C5040008E104000873
:1052BC0000000000000000000000000000000000E2
:1052CC000000000000000000000C0140010001047F
:1052DC00CD090008D90900089D0A0008790A0008C0
:1052EC00650A0008B90A0008DD0A0008120100026C
:1052FC000202004083044057000201020301000037
:10530C00040309041A030000000000000000000060
:10531C000000000000000000000000000000000081
:10532C00250B0008010B0008050B0008090B0008F1
:10533C0001000000100000000024F400C545000826
:10534C0083450008AD44000800000000D943000864
:10535C005F44000831440008000000000000000019
:10536C00000000000D440008014400081944000826
:10537C002544000809024300020100C03209040060
:10538C0000010202010005240010010524010001A6
:10539C0004240202052406000107058203080010FC
:1053AC0009040100020A0000000705010240000088
:1053BC00070581024000000009024300020100C001
:1053CC00320904000001020201000524001001054D
:1053DC0024010001042402020524060001070582B1
:1053EC000308001009040100020A0000000705016F
:1053FC000200020007058102000200000A060002FA
:10540C00000000400100000009074300020104C035
:10541C0032090400000102020100052400100105FC
:10542C002401000104240202052406000107058260
:10543C000308001009040100020A0000000705011E
:10544C00024000000705810240000000B00100206E
:10545C000000000000000000000000000000000040
:10546C000000000000000000000000000000000030
:10547C000000000000000000000000000000000020
:10548C000000000000000000000000000000000010
:10549C000000000000000000000000000000000000
:1054AC0000000000000000000000000000000000F0
:040000050800475553
:00000001FF
